:100000000C942A000C9447000C9447000C94470071
:100010000C9447000C9447000C9447000C94470044
:100020000C9447000C9447000C9447000C94470034
:100030000C9447000C9447000C9447000C94470024
:100040000C9447000C9447000C9447000C94470014
:100050000C94470011241FBECFE5D4E0DEBFCDBF16
:1000600010E0A0E6B0E0EEEBF0E002C005900D92EB
:10007000A036B107D9F710E0A0E6B0E001C01D92AC
:10008000A036B107E1F70E9449000C945D000C9482
:100090000000BB9A29E130E0C39A80E197E2F901C0
:1000A0003197F1F70197D9F7C39880E49CE9F901FA
:0E00B0003197F1F70197D9F7EFCFF894FFCF12
:00000001FF
